:020000040000FA
:02000000B8291D
:080008009818181218162C08B4
:10001000A0002D08A100A201A3010E280F28640052
:100020008C1A2B28FF30A207031CA307031CA00770
:10003000031CA107031C0800220F0D28230F0E2804
:10004000FA30A2000030A3000F28981818121816D2
:1000500064008C1E28281A080314B32904086400BD
:100060000C1E2F2899000314B329A401A501B31273
:10007000AE21031C0800D33E0319B3162D3EC63E25
:10008000031846280A3E031C38284D28F33E03185F
:100090003828063E031C38280A3EA2000430A3007C
:1000A000A20EA20DA40DA50DA30B5128A90303199F
:1000B0009A28AE21031C0800C63E031863280A3E96
:1000C000031C9A284D28F33E03189A28063E031C69
:1000D0009A280A3E4D28A401A501B312AE21031CA3
:1000E0000800D33E0319B3162D3EC63E03186E28F2
:1000F0000A3E031C6E28A2000310240DA000250D4B
:10010000A100200DA10DA4070318A10A2108A5072D
:10011000A40DA50D2208A4070318A50AA903031915
:100120009A28AE21031C0800C63E03189A280A3EEE
:1001300003187B28B31EA128A409A509A40A031942
:10014000A50A24080314B329B31329080319B31704
:100150000530A8002730A3001030BA200330A300D8
:10016000E830BA20A3016430BA20A3010A30BA20D3
:100170002408C128A2002508A1002408A00092217B
:100180002008A000A8030319B31329080319CB28DA
:100190002802031808002008031DB313B31B08002E
:1001A000303EAE290830A600A70037088400350885
:1001B00033192321331D2521360884008417340880
:1001C0008004A001A10126080319B329B31818213E
:1001D0003608840000083405FF3EA00DA10DB31CB5
:1001E0001821A60BE6282708331849292008B32927
:1001F0000830A60037088400350833192321331D41
:10020000252136088400841734098005260803193F
:10021000B3293318492136088400A10CA00C00082A
:100220003404031C340680001821A60B0B29B329C3
:10023000370884003508800600001E291F29202960
:1002400021298006080080042829FF3A80052929F1
:10025000FF3A84178005B329A301A200FF30A2074B
:10026000031CA307031CB3290330A100E6303A2185
:100270002E29A101FC3EA000A109031C4529FF3045
:100280000000A00703184029A0076400A10F3F2920
:100290000800A201A3015029A10CA00CA20DA30DDE
:1002A000FF3E03184C292308A1002208A000B3290F
:1002B0000310A00DA10DFF3E031858292008B329F3
:1002C0000310A10CA00CFF3E031860292008B329DD
:1002D000A101A301A20001307429A101A301A20080
:1002E00004307429A2000530A80023082102031D50
:1002F0007B29220820020430031801300319023040
:100300002805031DFF30B329A2002008A6002408F9
:10031000A0002608A4002108A6002508A1002608A0
:10032000A5009429A501A4011030A600210DA40D5B
:10033000A50D2208A4022308031C230FA5020318FD
:10034000A8292208A40723080318230FA5070310D0
:10035000A00DA10DA60B96292008B3298400310811
:100360008A0030088200831303138312640008009C
:100370008316203099002030980083129030980026
:10038000831607309F008117061086140611861108
:100390008312E90141308A012F2054308A012F2035
:1003A00034308A012F2035308A012F2020308A01F5
:1003B0002F2053308A012F2074308A012F20613082
:1003C0008A012F2072308A012F2074308A012F2059
:1003D00069308A012F206E308A012F2067308A0110
:1003E0002F202E308A012F202E308A012F202E30F0
:1003F0008A012F202E308A012F200D308A012F20D4
:100400000A308A012F20BE01BF01DE01C401C501EF
:10041000861583168611C83083128A012C218A1111
:100420000A1218238A110A120D2C8A110A128F221D
:1004300086118316861106308312B6000130B4008F
:100440000630B7000430B5000130B3005E08A000EC
:10045000A1018A01F8204408A0004508A10010303D
:100460008A01F9203808A0003908A1008A01F82083
:1004700064005E08683C8A110A120319462A640067
:100480005E08523C8A110A12031D5D2A0630B6002E
:100490000130B4000630B7000430B5000130B300BD
:1004A000A001A10110308A01F920A001A1011030A2
:1004B0008A01F9208A110A12792A64005E08563CE2
:1004C0008A110A1203196B2A64005E08543C8A11CF
:1004D0000A12031D792A0630B6000130B400063036
:1004E000B7000430B5000130B300A001A1018A01BA
:1004F000F82008003A08A0003B08A1003C08A4002E
:100500003D08A5000130A30008308A018421C600FF
:100510002108C7002408BE002508BF0008000310FA
:10052000C40DC50D39184414391C44103808B800DE
:10053000B9010800E801E201861183168611063030
:100540008312B6000130B4000630B7000430B500A5
:100550000130B3005730A000A1018A01F820063015
:10056000B6000230B4000630B7000430B5000230E7
:10057000B3008A01D220E700E80364006808003C69
:100580008A110A120319CC2A64008A110A12E71F81
:10059000AF2A8A110A12132B41308A012F205430BE
:1005A0008A012F2034308A012F2035308A012F20F4
:1005B00044308A012F2042308A012F2030308A01B6
:1005C0002F2034308A012F2031308A012F20203013
:1005D0008A012F2042308A012F2075308A012F2076
:1005E00073308A012F2079308A012F2020308A0130
:1005F0002F2045308A012F2072308A012F2072303F
:100600008A012F206F308A012F2072308A012F201B
:1006100021308A012F200D308A012F200A308A01D3
:100620002F200130E2008615831686118312080000
:1006300086118316861183125230DE00C401C50173
:10064000B801B9018A011522E40164002030640276
:100650008A110A1203183E2B0630B6000230B4008D
:100660000630B7000430B5000230B3008A01D22052
:10067000DD00E40A8A110A12031D252B8615831654
:100680008611831208008A019A2238306705C0005B
:10069000C1014008A0004108A10003308A01632184
:1006A000C0002108C100A001A1014108A300400829
:1006B0008A0172218A110A12031DA92B44308A0172
:1006C0002F2061308A012F2074308A012F20613061
:1006D0008A012F2046308A012F206C308A012F207A
:1006E00061308A012F2073308A012F2068308A01FF
:1006F0002F2020308A012F2053308A012F2069308B
:100700008A012F207A308A012F2065308A012F201C
:100710003D308A012F2035308A012F2031308A0167
:100720002F2032308A012F206B308A012F20623037
:100730008A012F2069308A012F2074308A012F20EE
:100740000D308A012F200A308A012F208A110A12C7
:10075000FF2B0130E3000130C0020030031C013EDA
:10076000C1026308A00040088A015B21E300443015
:100770008A012F2061308A012F2074308A012F20B6
:1007800061308A012F2046308A012F206C308A0187
:100790002F2061308A012F2073308A012F2068308A
:1007A0008A012F2020308A012F2053308A012F20E8
:1007B00069308A012F207A308A012F2065308A0122
:1007C0002F203D308A012F20A9016308A400A50134
:1007D0002E30B000B1018A01A4206D308A012F2093
:1007E00062308A012F2069308A012F2074308A01FB
:1007F0002F200D308A012F200A308A012F20080077
:100800005B08DE004608C4004708C5003E08B80083
:100810003F08B9008A011522080041308A012F20C3
:1008200074308A012F206D308A012F2065308A01B3
:100830002F206C308A012F2020308A012F20413058
:100840008A012F2054308A012F2034308A012F2032
:1008500035308A012F2044308A012F2042308A010E
:100860002F2030308A012F2034308A012F20313060
:100870008A012F2020308A012F2044308A012F2026
:1008800065308A012F206D308A012F206F308A0158
:100890002F200D308A012F200A308A012F203D3071
:1008A0008A012F203D308A012F203D308A012F20E0
:1008B0003D308A012F203D308A012F203D308A01B2
:1008C0002F203D308A012F203D308A012F203D30DE
:1008D0008A012F203D308A012F203D308A012F20B0
:1008E0003D308A012F203D308A012F203D308A0182
:1008F0002F203D308A012F203D308A012F203D30AE
:100900008A012F203D308A012F203D308A012F207F
:100910003D308A012F200D308A012F200A308A01B4
:100920002F208A0143230D308A012F200A308A01AB
:100930002F2041308A012F2074308A012F206D3002
:100940008A012F2065308A012F206C308A012F20E8
:1009500020308A012F2044308A012F2061308A0103
:100960002F2074308A012F2061308A012F204630D9
:100970008A012F206C308A012F2061308A012F20BC
:1009800073308A012F2068308A012F2020308A019D
:100990002F2044308A012F2065308A012F206D30AE
:1009A0008A012F206F308A012F200D308A012F20DD
:1009B0000A308A012F2057308A012F2061308A01A6
:1009C0002F2069308A012F2074308A012F2069304E
:1009D0008A012F206E308A012F2067308A012F2054
:1009E00020308A012F2066308A012F206F308A0143
:1009F0002F2072308A012F2020308A012F2064306E
:100A00008A012F2061308A012F2074308A012F2023
:100A100061308A012F202E308A012F202E308A014A
:100A20002F202E308A012F202E308A012F200D30CA
:100A30008A012F200A308A012F204F308A012F206F
:100A400070308A012F2074308A012F2069308A018A
:100A50002F206F308A012F206E308A012F207330B3
:100A60008A012F203A308A012F200D308A012F2051
:100A70000A308A012F2031308A012F2020308A014C
:100A80002F202D308A012F2020308A012F20523034
:100A90008A012F2065308A012F2061308A012F20A2
:100AA00064308A012F2020308A012F2066308A018D
:100AB0002F2072308A012F206F308A012F206D3055
:100AC0008A012F2020308A012F2061308A012F20B7
:100AD00064308A012F2064308A012F2072308A010D
:100AE0002F2065308A012F2073308A012F20733028
:100AF0008A012F200D308A012F200A308A012F20F1
:100B000032308A012F2020308A012F202D308A0197
:100B10002F2020308A012F2057308A012F20723059
:100B20008A012F2069308A012F2074308A012F20FA
:100B300065308A012F2020308A012F2074308A01ED
:100B40002F206F308A012F2020308A012F20613022
:100B50008A012F2064308A012F2064308A012F20DF
:100B600072308A012F2065308A012F2073308A016C
:100B70002F2073308A012F2020308A012F206530EA
:100B80008A012F2072308A012F2061308A012F20A4
:100B900073308A012F2065308A012F2020308A018E
:100BA0002F2066308A012F2069308A012F20723071
:100BB0008A012F2073308A012F2074308A012F2060
:100BC0000D308A012F200A308A012F2033308A010C
:100BD0002F2020308A012F202D308A012F20203015
:100BE0008A012F2057308A012F2072308A012F204E
:100BF00069308A012F2074308A012F2065308A01E4
:100C00002F2020308A012F2074308A012F206F304E
:100C10008A012F2020308A012F2061308A012F2065
:100C200064308A012F2064308A012F2072308A01BB
:100C30002F2065308A012F2073308A012F207330D6
:100C40008A012F2020308A012F206E308A012F2028
:100C50006F308A012F2020308A012F2065308A01D1
:100C60002F2072308A012F2061308A012F207330AB
:100C70008A012F2065308A012F200D308A012F2014
:100C80000A308A012F2034308A012F2020308A0137
:100C90002F202D308A012F2020308A012F2057301D
:100CA0008A012F2072308A012F2069308A012F207B
:100CB00074308A012F2065308A012F202F308A015D
:100CC0002F2052308A012F2065308A012F20613079
:100CD0008A012F2064308A012F2020308A012F20A2
:100CE00054308A012F2065308A012F2073308A0109
:100CF0002F2074308A012F2020308A012F2061306C
:100D00008A012F2074308A012F2020308A012F2061
:100D100061308A012F2064308A012F2064308A01DB
:100D20002F2072308A012F2065308A012F207330E6
:100D30008A012F2073308A012F200D308A012F2045
:100D40000A308A012F200D308A012F200A308A01B3
:100D50002F2041308A012F2064308A012F206430F7
:100D60008A012F2072308A012F2065308A012F20BE
:100D700073308A012F2073308A012F2020308A019E
:100D80002F206D308A012F2075308A012F2073307B
:100D90008A012F2074308A012F2020308A012F20D1
:100DA00062308A012F2065308A012F2020308A018D
:100DB0002F2061308A012F2020308A012F206430BB
:100DC0008A012F206F308A012F2075308A012F2051
:100DD00062308A012F206C308A012F2065308A0111
:100DE0002F2020308A012F2077308A012F206F306A
:100DF0008A012F2072308A012F2064308A012F202F
:100E000020308A012F2069308A012F206E308A011C
:100E10002F2020308A012F2068308A012F20653052
:100E20008A012F2078308A012F200D308A012F204F
:100E30000A308A012F2054308A012F2068308A011D
:100E40002F2065308A012F2020308A012F207E300C
:100E50008A012F2020308A012F2028308A012F205C
:100E600074308A012F2069308A012F206C308A016A
:100E70002F2064308A012F2065308A012F202930ED
:100E80008A012F2020308A012F2069308A012F20EB
:100E900073308A012F2020308A012F2075308A017B
:100EA0002F2073308A012F2065308A012F20643073
:100EB0008A012F2020308A012F2061308A012F20C3
:100EC00073308A012F2020308A012F2061308A015F
:100ED0002F2020308A012F2073308A012F20743078
:100EE0008A012F2061308A012F2072308A012F2041
:100EF00074308A012F202F308A012F2073308A010D
:100F00002F2074308A012F206F308A012F207030FB
:100F10008A012F2020308A012F2063308A012F2060
:100F20006F308A012F2064308A012F2065308A01BA
:100F30002F200D308A012F200A308A012F206630A1
:100F40008A012F206F308A012F206C308A012F20D8
:100F50006C308A012F206F308A012F2077308A0170
:100F60002F2065308A012F2064308A012F20203005
:100F70008A012F2062308A012F2079308A012F20A8
:100F800020308A012F2074308A012F2068308A0196
:100F90002F2065308A012F2020308A012F206F30CA
:100FA0008A012F2070308A012F2074308A012F206F
:100FB00069308A012F206F308A012F206E308A011C
:100FC0002F2020308A012F2061308A012F206E309F
:100FD0008A012F2064308A012F2020308A012F209F
:100FE00074308A012F2068308A012F2065308A01F1
:100FF0002F2020308A012F2061308A012F20643079
:101000008A012F2064308A012F2072308A012F201C
:1010100065308A012F2073308A012F2073308A01B6
:101020002F200D308A012F200A308A012F204530D1
:101030008A012F2078308A012F2061308A012F20E9
:101040006D308A012F2070308A012F206C308A0188
:101050002F2065308A012F203A308A012F2020303E
:101060008A012F207E308A012F2031308A012F20E3
:1010700030308A012F2030308A012F2030308A0111
:101080002F2034308A012F2032308A012F20303037
:101090008A012F2030308A012F2030308A012F2002
:1010A0000D308A012F200A308A012F2077308A01E3
:1010B0002F2069308A012F206C308A012F206C305C
:1010C0008A012F2020308A012F2072308A012F20A0
:1010D00065308A012F2061308A012F2064308A0117
:1010E0002F2020308A012F2064308A012F20613088
:1010F0008A012F2074308A012F2061308A012F202D
:1011000020308A012F2062308A012F2065308A0129
:101110002F2067308A012F2069308A012F206E30FE
:101120008A012F206E308A012F2069308A012F20FA
:101130006E308A012F2067308A012F2020308A01EB
:101140002F2061308A012F2074308A012F20203017
:101150008A012F2068308A012F2065308A012F20D4
:1011600078308A012F2020308A012F2030308A01E8
:101170002F2030308A012F2030308A012F20343048
:101180008A012F2032308A012F2030308A012F200F
:1011900030308A012F2030308A012F200D308A0113
:1011A0002F200A308A012F208A0125207E3C8A15B3
:1011B0000A12031DD4280130A9002530B000B10166
:1011C0008A016B20E5000430A9002530B000B10190
:1011D0008A013520BA002508BB000430A90025305B
:1011E000B000B1018A013520BC002508BD008A018C
:1011F0007A220A308A012F200D308A012F205030A8
:101200008A012F2061308A012F2067308A012F2028
:1012100065308A012F203A308A012F20A901460823
:10122000A4004708A5002E30B000B1018A01A42017
:1012300020308A012F2041308A012F2064308A011A
:101240002F2064308A012F2072308A012F203A30FB
:101250008A012F20A9013E08A4003F08A5002E30D6
:10126000B000B1018A01A4200D308A012F200A307C
:101270008A012F2064006508013C8A150A120319AF
:10128000852964006508023C8A150A120319362A6A
:1012900064006508033C8A150A120319362A6400A3
:1012A0006508043C8A150A120319F32A4F308A0193
:1012B0002F2070308A012F2074308A012F2069304E
:1012C0008A012F206F308A012F206E308A012F2053
:1012D00020308A012F2045308A012F2072308A0168
:1012E0002F2072308A012F206F308A012F20723018
:1012F0008A012F2021308A012F200D308A012F20D2
:101300000A308A012F208A01932C5230DE004608D1
:10131000C4004708C5003E08B8003F08B9008A016C
:1013200015220D308A012F200A308A012F205030DB
:101330008A012F2061308A012F2067308A012F20F7
:1013400065308A012F203A308A012F20A9014608F2
:10135000A4004708A5002E30B000B1018A01A420E6
:101360000D308A012F200A308A012F200130E4003D
:101370000630B6000230B4000630B7000430B500C5
:101380000230B3008A01D220DD00640080305D02AB
:101390008A150A12031CCE292E30DD00640020308D
:1013A0005D028A150A120318D7292E30DD005D0868
:1013B0008A012F20E40A8A150A12031DB82986150E
:1013C000831686110D3083128A012F200A308A017C
:1013D0002F204D308A012F206F308A012F2072304C
:1013E0008A012F2065308A012F203F308A012F206B
:1013F00020308A012F2031308A012F203D308A0190
:101400002F2079308A012F2065308A012F207330F8
:101410008A012F2020308A012F2032308A012F208C
:101420003D308A012F206E308A012F206F308A01D3
:101430002F200D308A012F200A308A012F20013001
:10144000A9002530B000B1018A016B20DD006400E5
:101450005D08013C8A110A12031D932CC60A031968
:10146000C70A8A150A1285298A01932C45308A01F8
:101470002F206E308A012F2074308A012F20653092
:101480008A012F2072308A012F2020308A012F20DC
:1014900074308A012F2065308A012F2078308A012C
:1014A0002F2074308A012F2020308A012F207E3097
:1014B0008A012F2020308A012F2028308A012F20F6
:1014C00074308A012F2069308A012F206C308A0104
:1014D0002F2064308A012F2065308A012F20293087
:1014E0008A012F2020308A012F2074308A012F207A
:1014F0006F308A012F2020308A012F2065308A0129
:101500002F206E308A012F2064308A012F200D3069
:101510008A012F200A308A012F208430DE003E0805
:10152000B8003F08B9008A011522E830AC0003304A
:10153000AD008A0104208A150A12031C952ADD00D9
:101540005D08A00020308A016D21C8005D08A00060
:101550007F308A016821CA0048084A048A150A12A5
:10156000031D952A64005D087E3C8A150A12031942
:10157000CB2A0630B6000130B4000630B700043084
:10158000B5000130B3005D08A000A1018A01F82078
:101590008A150A12952A861583168611640083120D
:1015A0006508023C8A150A12031DD82A8330DE0022
:1015B00064006508033C8A150A12031DE12A88307D
:1015C000DE004608C4004708C5008A0115228615BA
:1015D0008316861183128A019A2286158316861134
:1015E00083128A01932C57308A012F2072308A018E
:1015F0002F2069308A012F2074308A012F20693012
:101600008A012F206E308A012F2067308A012F2017
:1016100020308A012F2073308A012F2061308A0107
:101620002F206D308A012F2070308A012F206C30DE
:101630008A012F2065308A012F2020308A012F2037
:1016400074308A012F2065308A012F2078308A017A
:101650002F2074308A012F2020308A012F207430EF
:101660008A012F206F308A012F2020308A012F20FD
:1016700042308A012F2075308A012F2066308A017E
:101680002F2066308A012F2065308A012F2072308A
:101690008A012F2020308A012F2031308A012F200B
:1016A0003A308A012F20A9014608A4004708A50066
:1016B0002E30B000B1018A01A42020308A012F20F1
:1016C00061308A012F2074308A012F2020308A0156
:1016D0002F2041308A012F2064308A012F2064306E
:1016E0008A012F2072308A012F2065308A012F2035
:1016F00073308A012F2073308A012F203A308A01FB
:101700002F20A9013E08A4003F08A5002E30B000FC
:10171000B1018A01A4200D308A012F200A308A01EC
:101720002F208430DE003E08B8003F08B9008A014F
:1017300015223E30C200C301E4016408A000A101EB
:101740004308A30042088A016A218A150A12031D70
:10175000142C64083F3C8A150A12031CFD2B8A15C1
:101760000A12B623DD008A150A12FD2B0B308A00FF
:101770006408BD3E03188A0A8200573465346C340D
:1017800063346F346D346534213420345434683418
:1017900069347334203469347334203461346E34E2
:1017A0002034413474346D3465346C342034413425
:1017B00054343434353444344234303434343134B1
:1017C0004234203434346D34623469347434203417
:1017D000643461347434613466346C346134733429
:1017E0006834203438342034703469346E34203412
:1017F000633468346934703421340630B600013003
:10180000B4000630B7000430B5000130B3005D0805
:10181000A000A1018A01F8205D088A012F20E40AB6
:101820008A150A12031D9D2B8615831686110D300D
:1018300083128A012F200A308A012F2052308A0118
:101840002F2065308A012F2061308A012F206430DB
:101850008A012F2069308A012F206E308A012F20C3
:1018600067308A012F2020308A012F2062308A01C0
:101870002F2061308A012F2063308A012F206B30A6
:101880008A012F2020308A012F2062308A012F20E8
:1018900075308A012F2066308A012F2066308A0138
:1018A0002F2065308A012F2072308A012F202E30A0
:1018B0008A012F202E308A012F202E308A012F20DE
:1018C0000D308A012F200A308A012F205430DE008B
:1018D0003E08B8003F08B9008A011522E4016408F7
:1018E000A000A1014308A30042088A016A218A15C9
:1018F0000A12031D902C0630B6000230B4000630E8
:10190000B7000430B5000230B3008A01D220DD00F8
:101910005D088A012F20E40A8A150A12031D6F2C24
:101920008615831686110D3083128A012F200A3006
:101930008A012F2045308A012F2072308A012F2002
:1019400061308A012F2073308A012F2065308A018F
:101950002F2020308A012F2026308A012F2020308E
:101960008A012F2077308A012F2072308A012F20A0
:1019700069308A012F2074308A012F2065308A0156
:101980002F2020308A012F2074308A012F206F30C1
:101990008A012F2020308A012F2044308A012F20F5
:1019A00061308A012F2074308A012F2061308A0132
:1019B0002F2046308A012F206C308A012F20613081
:1019C0008A012F2073308A012F2068308A012F204E
:1019D00020308A012F2073308A012F2065308A0140
:1019E0002F2063308A012F2074308A012F206F301E
:1019F0008A012F2072308A012F202E308A012F2059
:101A00002E308A012F202E308A012F200D308A019E
:101A10002F200A308A012F208330DE004608C400C0
:101A20004708C5008A011522861583168611831280
:101A30008A019A22861583168611831252308A01F2
:101A40002F2065308A012F2061308A012F206430D9
:101A50008A012F2069308A012F206E308A012F20C1
:101A600067308A012F2020308A012F2062308A01BE
:101A70002F2061308A012F2063308A012F206B30A4
:101A80008A012F2020308A012F2044308A012F2004
:101A900061308A012F2074308A012F2061308A0141
:101AA0002F2046308A012F206C308A012F20613090
:101AB0008A012F2073308A012F2068308A012F205D
:101AC00020308A012F2073308A012F2065308A014F
:101AD0002F2063308A012F2074308A012F206F302D
:101AE0008A012F2072308A012F202E308A012F2068
:101AF0002E308A012F202E308A012F200D308A01AE
:101B00002F200A308A012F205230DE004608C40000
:101B10004708C5003E08B8003F08B9008A011522F1
:101B2000E4016408A000A1014308A30042088A015F
:101B30006A218A150A12031DB22D0630B600023042
:101B4000B4000630B7000430B5000230B3008A019B
:101B5000D220DD005D088A012F20E40A8A150A12CE
:101B6000031D912D8615831686110D3083128A016F
:101B70002F200A308A012F2046308A012F20693019
:101B80008A012F206E308A012F2069308A012F2090
:101B900073308A012F2068308A012F2065308A0136
:101BA0002F2064308A012F200D308A012F200A3027
:101BB0008A012F208A01932C64008A150A12DC2DD9
:081BC00063008A150A12E02DF2
:02400E00753FFC
:00000001FF
